:030000000219FDE5
:03000B000200AA46
:03002B0002019936
:03005B0002034C51
:0300730002033253
:1000800002030406080C10182030406080040608A3
:100090000C10182030406080A0C000070F1F3F0DDB
:1000A0000D04050D050305030302C2AF306308C24A
:1000B00063857C8AD2AF32C0D0C0E0206227E525BC
:1000C0006002E473E525F4C3334009758A00D26306
:1000D000F57C01D6F58A758B00758D00D262D0E073
:1000E000D0D0D2AF32C3E526334009758A00D2633F
:1000F000F57C01F6F58AC262E526F4603B306803C0
:10010000207213758B00758D00D0E0D0D0C292C2E2
:1001100096C294D2AF32C292C296C294206E0C2084
:100120006609740ED5E0FDE57E4290758B00758DF5
:1001300000D0E0D0D0D2AF32758A00D263757C0097
:10014000C28DD262212B01C4306805206602D29292
:1001500001C4306805206602D29401C430680520CD
:100160006602D29601C4C29330680A2066077410F2
:10017000D5E0FDD29201C4C29530680A20660774AA
:1001800010D5E0FDD29401C4C29730680A206607FA
:100190007410D5E0FDD29601C4C2AFC2AD53E6EFF4
:1001A000C0D0C0E0D2D3D2AFE57D6009E57A60056A
:1001B000757A0041DF757A01C2CEE52A60072074A6
:1001C00049152A410A7800790020742EE580307E96
:1001D00001F430E50278FF53DACF207E0343DA20C2
:1001E000307E0343DA10C2D8C271E580307E01F45C
:1001F00030E50279FFC3E89970CB306103752A18A6
:10020000207403752A18885FD27020740DE52B6066
:1002100004152B411A43DA01C2D82070024178A894
:100220005F206102C2702074367982B70431C3E85E
:1002300094F0400374F0F8E8C4540F28F87984B7B8
:100240000302415FC313C3138721200802C3132095
:100250000A06C3C898F8415F28F8500374FFF8886D
:1002600022E52D54066011E533C313C3132406257C
:1002700022F52250037522FF7882B6045985222484
:10028000A824C3E52495644002A864C3E8956640A9
:1002900002A8668825E569700241C9C3E8AA699A7F
:1002A0005003E8FAE4F9EAC333FBE56BF45B294059
:1002B0000D256AF8E56A6002156A400B41C90AC358
:1002C000E56A9A5002056A78FF8826C26EC3E52661
:1002D00094F84002D26EC3E52594404002D26420D7
:1002E000CF0AD0E0D0D043E610D2AD32C2CF053A2B
:1002F000E57D6009E57B6005757B006128757B0104
:100300007801E52A6005307402152AC3E55F94017F
:1003100040057562006128756300756C00E5622414
:1003200001F56250037562FFD0E0D0D043E610D2F1
:10033000AD32C2AFC0D053E67FC260759100855622
:1003400094855795759104D0D0D2AF32C2AF53E6A1
:10035000EFC2ADC0D0C0E0C0F0D2D3D2AFA8FBA9ED
:10036000FCE57D6007C3E913F9E813F8C2D83071E2
:100370000261BE53DACF207E0343DA10307E03439E
:10038000DA20D271E580307E01F420E502619588A3
:10039000278928A1EB53DACF207E0343DA20307E71
:1003A0000343DA10C2D8C271307402A1D77800E5D5
:1003B00080307E01F430E502A1D7885FA1BF53DA17
:1003C000CF207E0343DA20307E0343DA10C271204F
:1003D0006102819753DACF207E0343DA10307E0327
:1003E00043DA20C2D8D271885A895BC3E89558F89D
:1003F000E99559F97B007E087A00C3E8948CE9946A
:10040000005005755E008189882178A2E6A82160E8
:1004100055C3E894C8E994005008E4D2E4FB7A0A92
:100420008164C3E89468E994015008E4D2E3FB7A5C
:100430000F8164C3E894D0E994025008E4D2E2FB4F
:100440007A1E8164C3E894A0E994055008E4D2E1DF
:10045000FB7A3C8164C3E89498E994085008E4D29C
:10046000E0FB7A787E00C3E8955CFCE9955DFD30A1
:0F047000E70AECF42401FCEDF43400FD755E00A6
:10047F00C3EC9AED9E5003755E01885C895D855AC9
:10048F0058855B597802A1BFC3E89527F8E99528ED
:10049F00F9307C02A1A3307B02A1A3307A02A19C88
:1004AF0020750281BAE9FDE8FC81D9E9C313F9E8A7
:1004BF0013F8307902A19CE9C313F9E813F83078E7
:1004CF0002A19CE9C313FDE813FC20612CC3EC943B
:1004DF001CED9402400281F0ED701EC3EC94C850E5
:1004EF00180529E52970021529C3E529940A500238
:1004FF00A1D7755F00D270A1D7E5296002152978C1
:10050F0088E6F97400207F087896B90302789EE692
:10051F0024FAFEE43400FFC3EC9EFCED9FFD92082D
:10052F00B90310A2085007207609D276A14230767F
:10053F0002C276A2085016B9030DECF42401FCEDAB
:10054F00F43400FD02055C78007900A1A3B903150E
:10055F00EC33FCED33FDC3EC940AFCED9400FD503D
:10056F00047C007D00C3EC94FFED9400400678FFFF
:10057F007900A1A3EC8575F0A4C5F0A2F733F87943
:10058F000040030205BF78FF79000205BFE9C313DE
:10059F00F9E813F8307C0EE9600278FFC3E81338EE
:1005AF00F8E43400F9C3E894FFE99400400278FFBF
:1005BF00885FD270206102A1D7741FF4552F4BF5BD
:1005CF002FC274EB7002D274752A18307403752A17
:1005DF000A306102A1EB20740353DAFE2074037515
:1005EF002B06D0F0D0E0D0D0D2AD43E61032790157
:1005FF0002061B790302061B790A02061B791E02EB
:10060F00061B796402061B79C802061B7817E4D50E
:10061F00E0FDD8FAD9F6227A147B780206427A10D6
:10062F007B8C0206427A0D7BB40206427A0B7BC8A2
:10063F000206427902B27DE4C295D5E0FDD294D58F
:10064F00E0FDC294D5E0FDD295D5E0FDD292E576DE
:10065F00D5E0FDC2927496D5E0FDD9D9EAF8D5E080
:10066F00FDD8FBDBCEC29522C37C007D0075F00068
:10067F0005F0EA33FAEB33FB50F6EB13FBEA13FA10
:10068F00C3E9FFE8FEE89AF8E99BF95004EFF9EEA9
:10069F00F8B3EC33FCED33FDD5F0DFEDF9ECF822D8
:1006AF00E889F08A20D2D4F8A9F07B0030F70B7BD1
:1006BF00FFF42401F8E9F43400F9E88520F0A4AD43
:1006CF00F0F8E98520F0A4AFF0FEED2EF974003FAD
:1006DF00FA7C04C3EA13FAE913F9E813F8DCF48B94
:1006EF00F030F70AE8F42401F8E9F43400F9E88966
:1006FF00F0C2D4F8A9F0227882B60403020761C3CE
:10070F00E55F9401400302072B852224E4F545F5AC
:10071F0046F547F548F549C26D0207617882E6FC58
:10072F00D26DE522F523783879C7AA40AB41C3EBE8
:10073F0013FBEA13FAEC146013C3EB13FBEA13FA7F
:10074F00EC14146007C3EB13FBEA13FAD177884557
:10075F00894622C3E5459523F8E5469400F9500CE8
:10076F00C3E89480E994FF4016020792C3E8947F90
:10077F00E994005003020792787F7900020792787C
:10078F008079FF884A894B22E54A2547F8E54B35A2
:10079F0048F9854B20E4300701F43549FA30E70971
:1007AF00C3EA94F040150207D0C3EA940F50030236
:1007BF0007D078FF79FF7A0F0207D0780079007A97
:1007CF00F0C3E5249564500AC374019524500B02BD
:1007DF0007EEE54B20E70E0207EEE54B30E7068804
:1007EF004789488A492278A4E6FAC3E54A33F8E5EF
:1007FF004B33F91206AFE930E70BC3E89480E99465
:10080F00FF40130129C3E8947FE9940050020129A6
:10081F00787F79000129788079FFE820E715C3E513
:10082F002398F84009C3E894014003020850780167
:10083F00020850E8F424012523F8400302085078F9
:10084F00FF884C2278A5E6FAA848A9491206AFE915
:10085F0030E70CC3E89401E994FF4016020885C302
:0F086F00E894FFE99400500302088578FF7900B0
:10087E00020885780179FFE920E715C3E54C98F861
:10088E004009C3E8940140030208AC78010208ACA9
:10089E00E8F42401254CF840030208AC78FF8824C4
:1008AE002278FFC26420693D206A12D264C3E541FA
:1008BE00940A4009C3E52594405002C26479A1E729
:1008CE006023E541601F74FF8541F0848539F03067
:1008DE006A0375F005A4F8C5F0600278FFC3E895C9
:1008EE00675002A867886622C3E54094C8E5419424
:1008FE0000E5665003142107046002F56622020922
:10090E000F2275E890227883E6FFE5E820ECF7A841
:10091E00BDA9BE0573C3E57394084052757300E913
:10092E00FA79A0E76044EA7007E574601B02094A91
:10093E00C3E895746010E5745006600C14020956F5
:10094E000460F9020956E574F574C39472401B7580
:10095E0064C0C394044013756480C39404400B7543
:10096E006440C39404400375640075BB0822E564BB
:10097E002410500274FFF5647982B7040221A3C3D8
:10098E00A864E524985002A824C3E895664002A8FE
:10099E006688258826E573B4070375BB102274326A
:1009AE0079A687F0A4C5F0A2F733F8C3E8956440A2
:1009BE0002A86488228824882588268867227540A4
:1009CE00007541F022C2AF75C820A8CCA9CDAA3AB5
:1009DE0030CF010A75C824D2AFC3EA13FAE913F96E
:1009EE00E813F8AB3BAC3C883B893CC3E89BF8E989
:1009FE009C20690A547FF930670241F64153AD3DA0
:100A0E008A3DF9EA9D547FFA600478FF79FFAE3E85
:100A1E00AF3F8B3E8C3FC3EC9FFCC3E99CF542A8D5
:100A2E003BA93CC3E89EF8E99FF9C3E54113FBE5FA
:100A3E004013FAE82AF540E93BF54150067540FFB0
:100A4E007541FF419DAA40AB41AC40AD417E047F54
:100A5E0002C3EB940440021E1FC3EB940840021E17
:100A6E001FC3ED13FDEC13FCDEF7C3EA9CFAEB9DFE
:100A7E00FBEF6009C3E913F9E813F8DFF7EA28FA88
:100A8E00EB39FB8A408B4150067BFF8B408B41C379
:100A9E00EB94025002D2673069047F0341C878920A
:100AAE00E6FFC3E537948240110FC3E53794A040AB
:100ABE00010FC3EF940640027F057E03E541C45447
:100ACE000FF9E541C454F0F8E540C4540F28F8C3BB
:100ADE00E89EFAE99400FB4009C3EA9402EB940005
:100AEE0050047A02E4FB6142AA40AB41EBC4FEEA39
:100AFE00C4540F4EFCC3EA9CFAEB9400FBC3E813FC
:100B0E00C313F8EA28FAEB3400FB8A408B41C3EB9F
:100B1E0094024002C2677803EBC4FE7B00EAC45421
:100B2E000F4EFAC3EA98FA4005C3940250027A02B5
:100B3E007892E6FF3060026142855256855357D255
:100B4E006043E680C3E49AF8E49BF9C3E833F8E91E
:100B5E0033F930670261E3E8FAE9FBD3E913FDE804
:100B6E0013FC88528953C3EF94036038EF20E00DD5
:100B7E00E82CF8E93DF9ECFAEDFB020B9EE828F8BB
:100B8E00E939F9C3E82402F8E93400F97AFE7BFF6B
:100B9E00C3EF9403400E8A548B55884E894F8C5068
:100BAE008D518117885489558A4E8B4F8C508D519B
:100BBE00306920C3E53394034019E542A2E713F8E8
:100BCE00E555F4240138400B20E7087554FFF42452
:100BDE0001F5558117E8FAD3E813FC8852C3EF9458
:100BEE00036020EF20E007E82CF8ECFA8103E828F8
:100BFE002402F87AFEC3EF940340088A54884E8C80
:100C0E0050811788548A4E8C50E56BC33350026462
:100C1E006BF56B3060028121753404D26043E6803F
:100C2E00E52D5406601FA840A941C2AF53E67F755B
:100C3E009100C3E498F594E499F595759104D2600A
:100C4E0043E680D2AF22D265754400752000306B2A
:100C5E0003752040020C73D2657544007520403038
:0E0C6E006B03752000D2AF7801206722E52DC0
:100C7C0054066002C265C3E54194054013780294A2
:100C8C000540087803940540027806306902780A1A
:100C9C00206019E544601530690AC3E533940340BC
:100CAC0003D53406D2AFD26CA1569129D2AF000035
:100CBC00C2AF20672AE541C3FB940F40027B0FEBC8
:100CCC00240530730123306A02742820620123F951
:100CDC003069027982E58D13E58B13C39940B10518
:100CEC0044E59BF45440B52002A14030690A08C386
:100CFC00E8940A400108819C2065028173C2655307
:100D0C00E67F7591003067107594007595FC7591B0
:100D1C0004D26043E6808173AE40AF41C3EE33FE34
:100D2C00EF33FF50047EFF7FFFC3E49EF594E49FF6
:100D3C00F595A11AC3E53394025002817330650214
:100D4C008173D802A154819CC26C53E67F759100CB
:100D5C00855494855595759104854E56854F57D27B
:100D6C006043E680D2AFE52D54066008206A020588
:100D7C0033020D90306C0D206B0A20650715811520
:100D8C00810216212278003064053065027801E575
:100D9C003775F007A4F9E5F028F5F0E9A2F013A2F5
:100DAC00F113A2F213F537C394785003753778C357
:100DBC00E53795384008D266C292C296C29430602C
:100DCC0002A1CA855056855157D26043E680222035
:100DDC007D11C2AF754302C295D293D2AF759F40BD
:100DEC00020FAAC2AF754302C295D297D2AF759FBC
:100DFC0040020FAA307243207D20C2AF754303908E
:100E0C000177757E20C296C297306204D294C11EBF
:100E1C00D295D2AF759F41020FAAC2AF7543039012
:100E2C000177757E20C292C293306204D294C13E87
:100E3C00D295D2AF759F43020FAA207D17C2AF7512
:100E4C004303900152C296306202D294D2AF759F86
:100E5C0041020FAAC2AF754303900152C292306295
:100E6C0002D294D2AF759F43020FAA207D11C2AF5C
:100E7C00754304C293D297D2AF759F43020FAAC297
:100E8C00AF754304C297D293D2AF759F41020FAA9C
:100E9C00307243207D20C2AF754305900166757E8C
:100EAC0008C294C295306204D292C1BAD293D2AF26
:100EBC00759F40020FAAC2AF754305900188757EDD
:100ECC0080C294C295306204D296C1DAD297D2AF66
:100EDC00759F40020FAA207D17C2AF754305900184
:100EEC0048C294306202D292D2AF759F40020FAAD0
:100EFC00C2AF75430590015CC2943062EBD296D2BE
:100F0C00AF759F40020FAA207D11C2AF754306C278
:100F1C0097D295D2AF759F41020FAAC2AF75430607
:100F2C00C293D295D2AF759F43020FAA3072422062
:100F3C007D20C2AF754301900188757E80C292C23C
:100F4C0093306204D296E156D297D2AF759F43028A
:100F5C000FAAC2AF754301900166757E08C296C296
:100F6C0097306204D292E176D293D2AF759F41E171
:100F7C00AA207D16C2AF75430190015CC29230620B
:100F8C0002D296D2AF759F43E1AAC2AF75430190CE
:100F9C000148C296306202D292D2AF759F41C266AE
:100FAC0022900146757E00C292C296C294C293C230
:100FBC0097C295C262227880760908760908760471
:100FCC000876FF0876030876FF08760B0876030888
:100FDC007601087601788C76010876FF0876FF0892
:100FEC0076FF0876FF0876FF0876030876FF08760A
:100FFC00FF0876FF0876250876D008762808765004
:10100C000876040876FF08760208760008767A08D7
:10101C0076FF0876010876010876000876032278B8
:10102C0087E6FFC272BF0302D2727888E6C39403CC
:10103C006008C27DE630E102D27DC27E7889E6305E
:10104C00E102D27EC3EF94026008758E01D2730266
:10105C001063758E00C273227880E6149000809322
:0E106C0078A4F67881E6149000809378A5F6BB
:10107A007886E61490008D9378A6F6789CE6753803
:10108A00FF75390CB402067538A075390AB403061F
:10109A0075388275390578A3E61490009A93F56934
:1010AA00120FAD22227896E6FA7897E6FB7888E660
:1010BA00B40305C3EB940EFB307F047A007BFFC3B5
:1010CA00EB9AFCC3948250027C827575000575EC1C
:1010DA008575F0A4C3E5F0947D40F222D27F11AF6A
:1010EA0012060C7A007B007C10120602E55F2AFACF
:1010FA0074003BFBDCF37C04C3EB13FBEA13FADC5E
:10110A00F7FEC27F11AF22E5EF20E6037520000546
:10111A0020903FFFE520146006901FFF14600093A3
:10112A0004600375EF1253D9BF7581C043FF801263
:10113A0005FD75EF0243B203E5B3240420E70DF57C
:10114A0021E5E320E0068521B343E301120FAD75E3
:10115A0080FF75A40075F13075D4DF75900375A50D
:10116A00FC75F2FC75D50175A60175E241C292C201
:10117A0096C294120611D293D297D2951205FDC245
:10118A0093C297C295E4F8F6D8FD756B01120FC2A7
:10119A0012166B78988676753001C2AF120616124F
:1011AA00062612060C12062D12060C120634120618
:1011BA000CC2AF78FA79FA308507D9FBD8F7021C46
:1011CA0000112B116411AE11AF78988676120FAD0B
:1011DA0075A90075B680757D007588507589127578
:1011EA00C82475910475D84075A82275B80275E6A9
:1011FA0090759B80759D0075D10E75BCC075BB0836
:10120A0075BA1175E8801205FDD2AF12090C53DACE
:10121A00CF207E0343DA20307E0343DA1043DA011B
:10122A00C2D8C271120616D2617B037A0CE55E70CF
:10123A00077A0CDB030211BB12060C2070030211A1
:10124A00BBC270E55FC3940240E1E52F541F85617C
:10125A0060F561B560D5DAD5C26153DACF207E0375
:10126A0043DA20307E0343DA10C2D8C27178A2E68C
:10127A007008D274E52F54E0F52FC2757529001253
:10128A000611307409C3E529940A4002D275120680
:10129A000278023074027800C3E55F9840F0C2AF6A
:1012AA00120626120626120626D2AF120616754D09
:1012BA00007888E6B403026199120602788CE6C3C4
:1012CA0094015003021399E530C3940150030213A9
:1012DA0099207435C3E55F94FF5003021399C2AF96
:1012EA0012063BD2AF120611C3E55F940150EFC25A
:1012FA00AF120626120607120626D2AF120611C32D
:10130A00E55F94FF40E90218137F02D27F11AF1202
:10131A000611C2AFC27F11AFAE5FC3E55F947FD241
:10132A00AF40761205FDC2AF12063BD2AFDFDC1129
:10133A00E6C3EE94057897F61206161216AD121742
:10134A00967F0AD27F11AF120611C2AFC27F11AFC8
:10135A00AE5FC3E55F947FD2AF50E61205FDC2AF20
:10136A00120626120607120626D2AFDFD611E6EEBD
:10137A0024057896F61206161216AD1217C512062D
:10138A001111AFC3E55F94FF500241DB021813C38A
:10139A00E55F954D4003855F4D1206117801798806
:1013AA00E7B403027805C3E55F98400241BBC2AFC8
:1013BA0012063B12063B12063BD2AF1206167530D6
:1013CA0000E4F531F5320531E531F470390532784A
:1013DA009AE67819146012783214600D787D1460D8
:1013EA000878FA146003753200C3E532984017157D
:1013FA00327531B478998676C2AF12063BD2AF788D
:10140A00988676120611120607E52A7005307402CC
:10141A0021BB78012074027806C3E55F9840A7785B
:10142A0088E6C394036003120611E52A70030211C9
:10143A00BBC2AF120FADE4F522F523F524F525F56D
:10144A0026F56AD2AF7885E6C333F568E4F545F543
:10145A0046F547F548F549F573F52CF52DF5377539
:0D146A00730875BB101205FD120910E5E8AE
:1014770020ECFBA8BDA9BEE97001F8887412091415
:1014870075730875BB107887E6FE7602112B78878F
:10149700EEF6C2AF7564FF1209AC8522648522653A
:1014A700852266D2AF75220175240175250175263F
:1014B7000185636C756D0175B69075A903757D011E
:1014C7007888E6B40307C27D307602D27DD268D22F
:1014D70069753300120F13120F381209CC1209D392
:1014E7001209CC1209D31209CC0214FFC2AF112B77
:1014F700D2AF75730075BB08120C65120706120D83
:1015070091120DDB1209D3120C54306D03120762CE
:101517002067031208AF3067031208F6120D911205
:101527000E001209D3120C65306D03120797120DC6
:1015370091120E771209D3120C54306D031207F56E
:10154700120D91120E9C1209D3120C65306D031205
:101557000853120D91120F131209D3120910120C0E
:1015670054120D91120F381209141209D33069352C
:10157700206B3285676485676585636C756D017956
:10158700187A0CC3E53399400FC269D26A8A358548
:1015970067648567660215ACC3E55F940140030283
:1015A70014FF021629306A1B206B18E535147004E6
:1015B700C26A81F3F535C3E55F940140030214FF66
:1015C700021629753600C3E56278FA9850543074CC
:1015D70004E52A604D7888E6B40317207D05207658
:1015E70007A1F9307602A1F9206B07D26B856764F2
:1015F700A13E78F0306B058567647820C3E5419894
:10160700500281FF306B1BC26BC27D307602D27DE8
:10161700D26A75351285676481FF0536E55F60021A
:10162700C12C753600C2AF120FAD7887E6FE760281
:10163700112B7887EEF6E4F522F523F524F525F549
:1016470026F568C26875A90075B680757D00D2AFAA
:101657001205FD120FAD307409C3E536940540023B
:1016670021BB61CB901A0D78201216EFE520B455F7
:101677000CA31216EFE520B4AA0302168D120FC2AF
:101687001216AD0216AC901A0378807B0A1216EF79
:10169700A308DBF9901A0F788C7B181216EFA308B2
:1016A700DBF9901A2722C2AF12172E121708901AC9
:1016B70000740E1216F4A374041216F4A374141211
:1016C70016F4901A0378807B0A1216F3A308DBF945
:1016D700901A0F788C7B181216F3A308DBF91217F0
:1016E7004112171F901A2722E493F622E6438F012F
:1016F700538FFD75EF0275B7A575B7F1F0538FFEE0
:1017070022438F02438F0175EF0275B7A575B7F1B5
:10171700901A0DF0538FFC22901A0D7455D1F49046
:101727001A0E74AAD1F4227A3079D07820901A4010
:10173700D1EFE520F709A3DAF7227A3079D0901AAA
:1017470040E7D1F409A3DAF922AB77A878BB010205
:101757007980BB02027981BB03027982BB040279DB
:1017670084BB05027986BB06027992BB070279879B
:10177700BB080279A3BB0902799CBB0A027988BB23
:101787000B027989E8F7227C05120616DCFB22C2D8
:10179700AF12062612062D12063412063B12060752
:1017A70012062612062D12063412063B12060712DF
:1017B700062612062D12063412063BD2AF22C2AFFE
:1017C70012063B12063412062D12062612060712BF
:1017D700063B12063412062D1206261206071206BB
:1017E7003B12063412062D120626D2AF22AE77AF71
:1017F70078C2AF120626120626120626120607DE42
:10180700F212063B120607DFF8D2AF221217961222
:10181700178E12178E757701757801757900121773
:10182700F47C05AD5F120616C3ED955F70F5C3E551
:101837005F9401400AC3E55F94FF403702185712CF
:1018470017501216AD121796C2AF75EF1212178EF8
:10185700DCD10579C3E5799403500280C112178E54
:0F1867000578E5771490009F93F808C3E578980B
:10187600500280A812178E12178E0577C3E577944B
:101886000C50028094120FC21216ADC2AF75EF1241
:0318960012178E98
:0319FD00021111C3
:101A00000E0414090904FF03FF0B03010155AA0189
:101A1000FFFFFFFFFF03FFFFFF25D0285004FF0259
:081A2000007AFF01010003FF41
:101A400023544253437562653132412320202020C4
:101A500023424C48454C492346333930232020202B
:101A60002020202020202020202020202020202076
:101C0000C2AFC2D353D9BF7581C043B20343FF8073
:101C1000752438752503B1C975EF0275E24043F1AB
:101C20002053A4DF75D400D2857DFA780379E67C51
:101C300010752200752300901DD67B0675249875BB
:101C400025013085028142208508D8FBD9F9DCF7CF
:101C500081B4308508D8FBD9F9DCF781B4B189E4C7
:101C600093A3C39A6004DDC381B4DBDBB17B600264
:101C7000812B7B08E493FAA3B15CDBF87A30B15C8A
:101C8000752200752300B17BEAFCEBFDC3ED94FEE9
:101C9000400EB17B8A278B28ED30E0048A828B834B
:101CA000B17B7AC270D8C3ED94FE601350CEBD00F4
:101CB00025EC60097520007521FF0200008100A855
:101CC00027A9280809D804D90281D3B17FEA89AAB3
:101CD000F281C50D81A0C3ED94035049EDA2E092BD
:101CE000007AC5C3E5829400E583941C50902000DF
:101CF00010438F02438F0175B7A575B7F1F030001F
:101D00001FA827A9280809438F01538FFDD804D99C
:101D100002A12089AAE275B7A575B7F1F0A3A10DBC
:101D2000538FFC817C7AC1BD030CE493A3FAB140CC
:101D3000DCF8B138817C817EAA22AB23B15CEBFA5E
:101D4000EA6222752608C3E52313F523E52213F57D
:101D50002250066323A0632201D526EAB1C9B1C986
:101D600075260AEAF4200102D285300102C285B14B
:101D7000C9C3134002C201D526EB22B17FEAFB2082
:101D80008502A17F308502A184752608AE24AF2587
:101D9000C3EF13FFEE13FEB1CDB1C9C3EA13308513
:101DA000024480FA30E703632201C3E52313F523DD
:101DB000E52213F52250066323A0632201D526D91C
:101DC000E52265236523F52222AE24AF250E0FDE22
:101DD000FEDFFCD20122424C48656C693437316326
:041DE000F390060175
:00000001FF
